Microchip MPLAB XC8 Compiler V2.32

Linker command line:

-W-3 --edf=C:\Program Files\Microchip\xc8\v2.32\pic\dat\en_msgs.txt -cn \
  -h+dist/default/production\LCD_Switch.X.production.sym \
  --cmf=dist/default/production\LCD_Switch.X.production.cmf -z -Q18F4580 \
  -oC:\Users\Dell7270\AppData\Local\Temp\xcAs7ac.4 --defsym=__MPLAB_BUILD=1 \
  -Mdist/default/production/LCD_Switch.X.production.map -E1 \
  -ver=XC8 Compiler --acfsm=1493 -ASTACK=071h-05FFh -pstack=STACK \
  -ACODE=01400h-07F00h -ACONST=01400h-07F00h \
  -ASMALLCONST=01400h-014FFhx107,07F00h-07F00h -AMEDIUMCONST=01400h-07F00h \
  -ACOMRAM=01h-05Fh -AABS1=00h-05FFh -ABIGRAM=01h-05FFh \
  -ARAM=060h-0FFh,0100h-01FFhx5 -ABANK0=060h-0FFh -ABANK1=0100h-01FFh \
  -ABANK2=0200h-02FFh -ABANK3=0300h-03FFh -ABANK4=0400h-04FFh \
  -ABANK5=0500h-05FFh -ASFR=0D00h-0DFFhx2,0F00h-0F5Fh,0F60h-0FFFh \
  -ACONFIG=0300000h-030000Dh -AIDLOC=0200000h-0200007h \
  -AEEDATA=0F00000h-0F000FFh -peeprom_data=EEDATA \
  -preset_vec=00h,intcode,intcodelo,powerup,init -pramtop=0600h \
  -psmallconst=SMALLCONST -pmediumconst=MEDIUMCONST -pconst=CONST \
  -AFARRAM=00h-00h \
  -prdata=COMRAM,nvrram=COMRAM,nvbit=COMRAM,rbss=COMRAM,rbit=COMRAM \
  -pfarbss=FARRAM,fardata=FARRAM,nvFARRAM=FARRAM \
  -pintsave_regs=BIGRAM,bigbss=BIGRAM,bigdata=BIGRAM -pbss=RAM \
  -pidata=CODE,irdata=CODE,ibigdata=CODE,ifardata=CODE -prparam=COMRAM \
  C:\Users\Dell7270\AppData\Local\Temp\xcAs7ac.o \
  dist/default/production\LCD_Switch.X.production.o 

Object code version is 3.11

Machine type is 18F4580



                Name                               Link     Load   Length Selector   Space Scale
C:\Users\Dell7270\AppData\Local\Temp\xcAs7ac.o
                idloc                            200000   200000        8        0       5
                config                           300000   300000        E        0       4
                init                                  0        0        4        0       0
dist/default/production\LCD_Switch.X.production.o
                idloc                            200000   200000        8        0       5
                config                           300000   300000        E        0       4
                text4                              7D90     7D90       30     3EC8       0
                text3                              7D6A     7D6A       26     3EB5       0
                text2                              7D2E     7D2E       1A     3E97       0
                text1                              7DC0     7DC0       30     3EE0       0
                text0                              7E36     7E36       CA     3F1B       0
                cstackCOMRAM                          1        1       3B        1       1
                dataBANK0                            60       60       11       60       1
                dataCOMRAM                           3C       3C       22        1       1
                cinit                              7DF0     7DF0       46     3EF8       0
                idataBANK0                         7D1D     7D1D       11     7D1D       0
                idataCOMRAM                        7D48     7D48       22     7D48       0

TOTAL           Name                               Link     Load   Length     Space
        CLASS   STACK          

        CLASS   CODE           
                init                                  0        0        4         0
                text4                              7D90     7D90       30         0
                text3                              7D6A     7D6A       26         0
                text2                              7D2E     7D2E       1A         0
                text1                              7DC0     7DC0       30         0
                text0                              7E36     7E36       CA         0
                cinit                              7DF0     7DF0       46         0
                idataBANK0                         7D1D     7D1D       11         0
                idataCOMRAM                        7D48     7D48       22         0

        CLASS   CONST          

        CLASS   SMALLCONST     

        CLASS   MEDIUMCONST    

        CLASS   COMRAM         
                cstackCOMRAM                          1        1       3B         1
                dataCOMRAM                           3C       3C       22         1

        CLASS   ABS1           

        CLASS   BIGRAM         

        CLASS   RAM            

        CLASS   BANK0          
                dataBANK0                            60       60       11         1

        CLASS   BANK1          

        CLASS   BANK2          

        CLASS   BANK3          

        CLASS   BANK4          

        CLASS   BANK5          

        CLASS   SFR            

        CLASS   CONFIG         
                config                           300000   300000        E         4

        CLASS   IDLOC          
                idloc                            200000   200000        8         5

        CLASS   EEDATA         

        CLASS   FARRAM         



SEGMENTS        Name                           Load    Length   Top    Selector   Space  Class

                reset_vec                      000000  000004  000004         0       0  CODE    
                cstackCOMRAM                   000001  00005D  00005E         1       1  COMRAM  
                dataBANK0                      000060  000011  000071        60       1  BANK0   
                idataBANK0                     007D1D  000011  007D2E      7D1D       0  CODE    
                text2                          007D2E  00001A  007D48      3E97       0  CODE    
                idataCOMRAM                    007D48  000022  007D6A      7D48       0  CODE    
                text3                          007D6A  000026  007D90      3EB5       0  CODE    
                text4                          007D90  000030  007DC0      3EC8       0  CODE    
                text1                          007DC0  000030  007DF0      3EE0       0  CODE    
                cinit                          007DF0  000046  007E36      3EF8       0  CODE    
                text0                          007E36  0000CA  007F00      3F1B       0  CODE    


UNUSED ADDRESS RANGES

        Name                Unused          Largest block    Delta
        BANK0            000071-0000FF               8F
        BANK1            000100-0001FF              100
        BANK2            000200-0002FF              100
        BANK3            000300-0003FF              100
        BANK4            000400-0004FF              100
        BANK5            000500-0005FF              100
        BIGRAM           00005E-00005F                2
                         000071-0005FF              58F
        CODE             001400-007D1C             691D
                         007F00-007F00                1
        COMRAM           00005E-00005F                2
        CONST            001400-007D1C             691D
                         007F00-007F00                1
        EEDATA           F00000-F000FF              100
        MEDIUMCONST      001400-007D1C             691D
                         007F00-007F00                1
        RAM              000071-0005FF              100
        SFR              000D00-000FFF              100
        SMALLCONST       001400-007D1C              100
                         007F00-007F00                1
        STACK            000071-0005FF              58F

                                  Symbol Table

_PORTD                   (abs)        000F83
_RB5                     (abs)        007C0D
_RC0                     (abs)        007C10
_RC1                     (abs)        007C11
_RC2                     (abs)        007C12
_RC3                     (abs)        007C13
_TRISB                   (abs)        000F93
_TRISC                   (abs)        000F94
_TRISD                   (abs)        000F95
__HRAM                   (abs)        000000
__Habs1                  abs1         000000
__Hbank0                 bank0        000000
__Hbank1                 bank1        000000
__Hbank2                 bank2        000000
__Hbank3                 bank3        000000
__Hbank4                 bank4        000000
__Hbank5                 bank5        000000
__Hbigbss                bigbss       000000
__Hbigdata               bigdata      000000
__Hbigram                bigram       000000
__Hbss                   bss          000000
__Hcinit                 cinit        000000
__Hclrtext               clrtext      000000
__Hcomram                comram       000000
__Hconfig                config       30000E
__Hconst                 const        000000
__HcstackCOMRAM          cstackCOMRAM 000000
__Hdata                  data         000000
__HdataBANK0             dataBANK0    000000
__HdataCOMRAM            dataCOMRAM   000000
__Heeprom_data           eeprom_data  000000
__Hfarbss                farbss       000000
__Hfardata               fardata      000000
__Hibigdata              ibigdata     000000
__Hidata                 idata        000000
__HidataBANK0            idataBANK0   000000
__HidataCOMRAM           idataCOMRAM  000000
__Hidloc                 idloc        200008
__Hifardata              ifardata     000000
__Hinit                  init         000004
__Hintcode               intcode      000000
__Hintcode_body          intcode_body 000000
__Hintcodelo             intcodelo    000000
__Hintentry              intentry     000000
__Hintret                intret       000000
__Hintsave_regs          intsave_regs 000000
__Hirdata                irdata       000000
__Hmediumconst           mediumconst  000000
__HnvFARRAM              nvFARRAM     000000
__Hnvbit                 nvbit        000000
__Hnvrram                nvrram       000000
__Hparam                 rparam       000000
__Hpowerup               powerup      000000
__Hram                   ram          000000
__Hramtop                ramtop       000600
__Hrbit                  rbit         000000
__Hrbss                  rbss         000000
__Hrdata                 rdata        000000
__Hreset_vec             reset_vec    000000
__Hrparam                rparam       000000
__Hsfr                   sfr          000000
__Hsmallconst            smallconst   000000
__Hspace_0               (abs)        007F00
__Hspace_1               (abs)        000071
__Hspace_2               (abs)        000000
__Hspace_4               (abs)        60000E
__Hstack                 stack        000000
__Hstruct                struct       000000
__Htemp                  temp         000000
__Htext                  text         000000
__Htext0                 text0        000000
__Htext1                 text1        000000
__Htext2                 text2        000000
__Htext3                 text3        000000
__Htext4                 text4        000000
__LRAM                   (abs)        000001
__Labs1                  abs1         000000
__Lbank0                 bank0        000000
__Lbank1                 bank1        000000
__Lbank2                 bank2        000000
__Lbank3                 bank3        000000
__Lbank4                 bank4        000000
__Lbank5                 bank5        000000
__Lbigbss                bigbss       000000
__Lbigdata               bigdata      000000
__Lbigram                bigram       000000
__Lbss                   bss          000000
__Lcinit                 cinit        000000
__Lclrtext               clrtext      000000
__Lcomram                comram       000000
__Lconfig                config       000000
__Lconst                 const        000000
__LcstackCOMRAM          cstackCOMRAM 000000
__Ldata                  data         000000
__LdataBANK0             dataBANK0    000000
__LdataCOMRAM            dataCOMRAM   000000
__Leeprom_data           eeprom_data  000000
__Lfarbss                farbss       000000
__Lfardata               fardata      000000
__Libigdata              ibigdata     000000
__Lidata                 idata        000000
__LidataBANK0            idataBANK0   000000
__LidataCOMRAM           idataCOMRAM  000000
__Lidloc                 idloc        000000
__Lifardata              ifardata     000000
__Linit                  init         000000
__Lintcode               intcode      000000
__Lintcode_body          intcode_body 000000
__Lintcodelo             intcodelo    000000
__Lintentry              intentry     000000
__Lintret                intret       000000
__Lintsave_regs          intsave_regs 000000
__Lirdata                irdata       000000
__Lmediumconst           mediumconst  000000
__LnvFARRAM              nvFARRAM     000000
__Lnvbit                 nvbit        000000
__Lnvrram                nvrram       000000
__Lparam                 rparam       000000
__Lpowerup               powerup      000000
__Lram                   ram          000000
__Lramtop                ramtop       000600
__Lrbit                  rbit         000000
__Lrbss                  rbss         000000
__Lrdata                 rdata        000000
__Lreset_vec             reset_vec    000000
__Lrparam                rparam       000000
__Lsfr                   sfr          000000
__Lsmallconst            smallconst   000000
__Lspace_0               (abs)        000000
__Lspace_1               (abs)        000000
__Lspace_2               (abs)        000000
__Lspace_4               (abs)        000000
__Lstack                 stack        000000
__Lstruct                struct       000000
__Ltemp                  temp         000000
__Ltext                  text         000000
__Ltext0                 text0        000000
__Ltext1                 text1        000000
__Ltext2                 text2        000000
__Ltext3                 text3        000000
__Ltext4                 text4        000000
__S0                     (abs)        007F00
__S1                     (abs)        000071
__S2                     (abs)        000000
__S4                     (abs)        000000
__S5                     (abs)        000000
___inthi_sp              stack        000000
___intlo_sp              stack        000000
___param_bank            (abs)        000000
___rparam_used           (abs)        000001
___sp                    stack        000000
__accesstop              (abs)        000060
__activetblptr           (abs)        000000
__end_of__initialization cinit        007E30
__end_of_command         text3        007D90
__end_of_data            text2        007D48
__end_of_delay           text4        007DC0
__end_of_display         text1        007DF0
__end_of_main            text0        007F00
__initialization         cinit        007DF0
__mediumconst            mediumconst  000000
__pcinit                 cinit        007DF0
__pcstackCOMRAM          cstackCOMRAM 000001
__pdataBANK0             dataBANK0    000060
__pdataCOMRAM            dataCOMRAM   00003C
__pidataBANK0            idataBANK0   007D1D
__pidataCOMRAM           idataCOMRAM  007D48
__ptext0                 text0        007E36
__ptext1                 text1        007DC0
__ptext2                 text2        007D2E
__ptext3                 text3        007D6A
__ptext4                 text4        007D90
__ramtop                 ramtop       000600
__size_of_command        (abs)        000000
__size_of_data           (abs)        000000
__size_of_delay          (abs)        000000
__size_of_display        (abs)        000000
__size_of_main           (abs)        000000
__smallconst             smallconst   000000
_command                 text3        007D6A
_data                    text2        007D2E
_delay                   text4        007D90
_display                 text1        007DC0
_main                    text0        007E36
command@a                cstackCOMRAM 000006
data@b                   cstackCOMRAM 000006
delay@i                  cstackCOMRAM 000004
delay@ms                 cstackCOMRAM 000001
display@p                cstackCOMRAM 000007
end_of_initialization    cinit        007E30
intlevel0                text         000000
intlevel1                text         000000
intlevel2                text         000000
intlevel3                text         000000
isa$std                  (abs)        000001
isa$xinst                (abs)        000000
main@F10470              dataCOMRAM   00004D
main@F10472              dataCOMRAM   00003C
main@F10474              dataBANK0    000060
main@arr                 cstackCOMRAM 000009
main@arr1                cstackCOMRAM 00001A
main@arr2                cstackCOMRAM 00002B
stackhi                  (abs)        0005FF
stacklo                  (abs)        000071
start                    init         000000
start_initialization     cinit        007DF0


MODULE INFORMATION

Module		Function		Class		Link	Load	Size
LCD switch.c
		_delay         		CODE           	7D90	0000	48
		_display       		CODE           	7DC0	0000	48
		_main          		CODE           	7E36	0000	202
		_data          		CODE           	7D2E	0000	26
		_command       		CODE           	7D6A	0000	38

LCD switch.c estimated size: 362

shared
		__initialization		CODE           	7DF0	0000	64

shared estimated size: 64

